:1000000012C02CC02BC02AC029C028C027C026C0BF
:1000100025C090C123C022C021C020C020C01EC066
:100020001DC01CC01BC011241FBECFE5D4E0DEBF25
:10003000CDBF10E0A0E6B0E0E8E2F7E002C0059036
:100040000D92AE36B107D9F710E0AEE6B0E001C0D0
:100050001D92A638B107E1F720D064C3D1CF1F921B
:100060000F920FB60F9211248F939F93AF93BF936C
:1000700084B195B1A0E0B0E080936E0090936F00E2
:10008000A0937000B0937100BF91AF919F918F9139
:100090000F900FBE0F901F901895BF92CF92DF92D6
:1000A000EF92FF920F931F93CF93DF9382E087BB72
:1000B00018BA3BD2A5D283B7856083BF89B7816068
:1000C00089BF12BE86B18F6E86B93E9A80E29EE4E9
:1000D0000197F1F781E01DD280EA9FE00197F1F7E7
:1000E000789424E6B22E94E6C92ED12C0CE91FEFA9
:1000F00088ECE82EF12CADD280936D00813041F474
:1001000084B195B1029790937300809372002AC0D6
:100110008230A9F4609178007091790080917A0022
:1001200090917B002AE030E040E050E09AD224E653
:1001300030E040E050E0D4D220936C0013C0833014
:1001400031F480916A0090916B00059607C084306D
:1001500049F480916A0090916B00059790936B0031
:1001600080936A0080916A0090916B00885E934052
:1001700020F010926B0010926A00809176009091AE
:100180007700C0916A00D0916B008C179D0708F032
:10019000C19A80917600909177008C179D0708F4A2
:1001A000C19860916E0070916F0080917000909185
:1001B0007100209172003091730040E050E0621BAA
:1001C000730B840B950B24EF31E040E050E049D2F3
:1001D0002FEF33E040E050E083D2C901DA01809391
:1001E000780090937900A0937A00B0937B0060919F
:1001F00078007091790080917A0090917B0024E6DC
:1002000030E040E050E06CD2209380008091780094
:1002100090917900A0917A00B0917B0020918000AC
:100220002B9D90011124821B8093810060917800A6
:100230007091790080917A0090917B002AE030E003
:1002400040E050E00ED220916C0030E040E050E001
:1002500047D230937700209376008091760090917A
:10026000770064E670E028D26093820020917600E7
:100270003091770080918200809F802D1124820F21
:1002800080938300D0937D00C0937C00CE0164E610
:1002900070E012D270938500609384006C9DC00161
:1002A0006D9D900D7C9D900D1124C81BD90BD09392
:1002B0007F00C0937E0080E82CD180916E009091E9
:1002C0006F00A0917000B091710057D085E821D1E6
:1002D00080918000F5D08EE222D180918100DCD027
:1002E00086E51DD18BE815D180E519D18091840078
:1002F000E7D08EE214D180917E00CED080EC09D17F
:1003000080E690E042D18DE30AD180918200D8D07E
:100310008EE205D180918300BFD080E200D185E6D6
:1003200090E033D188E893E1F7013197F1F7019735
:10033000D9F7E1CE1F920F920FB60F9211242F938F
:100340003F934F935F936F937F938F939F93AF935D
:10035000BF93EF93FF935BD1FF91EF91BF91AF916B
:100360009F918F917F916F915F914F913F912F91CD
:100370000F900FBE0F901F901895EF92FF920F9362
:100380001F939C0168EE73E097D1182F092FC901C4
:1003900068EE73E091D1662311F480E302C0862FEA
:1003A000805DBDD0812F902F64E670E085D1F82E5E
:1003B000E92E812F902F64E670E07ED1662311F440
:1003C00080E302C0862F805DAAD08F2D9E2D6AE02B
:1003D00070E072D1362F8F2D9E2D6AE070E06CD1C7
:1003E000182F332311F480E302C0832F805D97D050
:1003F000812F805D94D01F910F91FF90EF90089511
:100400000F931F939C0164E670E056D1182F092FBB
:10041000C90164E670E050D1662311F480E302C0A4
:10042000862F805D7CD0812F902F6AE070E044D1D0
:10043000362F812F902F6AE070E03ED1182F3323A2
:1004400011F480E302C0832F805D69D0812F805D2D
:1004500066D01F910F9108951F93282F64E620D135
:10046000192F822F1DD1882311F480E301C0805DF4
:1004700056D0812F6AE014D1282F812F11D1192F46
:10048000222311F480E302C0822F805D48D0812FA7
:10049000805D45D01F9108951F93282F6AE000D1F9
:1004A000382F822FFDD0192F332311F480E302C09F
:1004B000832F805D34D0812F805D31D01F910895CE
:1004C000805D2DD008959AE69A95F1F7909892B3B1
:1004D000807F9F70982B92BB929A85E08A95F1F766
:1004E0009298089592B3282F207F9F70292B22BBCA
:1004F000929A25E0922F9A95F1F7929892B382956D
:10050000807F9F70982B92BB929A2A95F1F79298D0
:1005100008959AE69A95F1F79098E4DF08959AE69F
:100520009A95F1F7909ADEDF08950F931F9381B3A8
:10053000806F81BB889A899A8A9A80E991E028EC39
:1005400030E0F9013197F1F70197D9F780E3BBDF8C
:1005500080E29EE40197F1F780E3B5DF00EA1FE057
:10056000C8010197F1F780E3AEDF88E2ACDF88E2F3
:10057000D0DF8CE0CEDF81E0CCDFC8010197F1F75E
:1005800086E0C7DF1F910F910895CF93DF93EC01B1
:1005900002C02196C4DF88818823D9F7DF91CF91EB
:1005A0000895CF93DF93EC0104C0FE01849121965E
:1005B000B6DF88818823C9F7DF91CF9108950F9323
:1005C0001F93CF93DF938C01862F90E087709070FC
:1005D00023E0880F991F2A95E1F780649ADFC0E035
:1005E000D0E0F801EC0FFD1FE4918E2F98DF2196EB
:1005F000C830D105B1F7DF91CF911F910F910895C8
:1006000087B3837C87BB88B38C6388BB0895B59917
:1006100002C091E00BC0B39902C093E007C0B49947
:1006200002C092E003C0B29911C094E080917500BD
:10063000873420F08EE38093750005C08F5F809330
:100640007500843029F49093740008951092750019
:10065000089580917400109274000895809374003E
:100660000895629FD001739FF001829FE00DF11DFC
:10067000649FE00DF11D929FF00D839FF00D749F1C
:10068000F00D659FF00D9927729FB00DE11DF91FC8
:10069000639FB00DE11DF91FBD01CF011124089525
:1006A000991B79E004C0991F961708F0961B881FC4
:1006B0007A95C9F780950895AA1BBB1B51E107C025
:1006C000AA1FBB1FA617B70710F0A61BB70B881FE2
:1006D000991F5A95A9F780959095BC01CD01089571
:1006E000A1E21A2EAA1BBB1BFD010DC0AA1FBB1F36
:1006F000EE1FFF1FA217B307E407F50720F0A21BA8
:10070000B30BE40BF50B661F771F881F991F1A9414
:1007100069F760957095809590959B01AC01BD013E
:08072000CF010895F894FFCF0A
:0E072800416C6B2E006D672F6C00C80004043E
:00000001FF
